:1000000011308A00D2290000FF00030E8301A100F5
:100010000A08A0008A010408A2007708A300780853
:10002000A4007908A5007A08A60003170D08031399
:10003000A70003170F080313A80003170C080313E6
:10004000A90003170E080313AA00831383128C3030
:100050008400801E2D288C1A58288C308400001CA7
:1000600033280C185B288B1E37280B195E282208B2
:1000700084002308F7002408F8002508F900260862
:10008000FA00270803178D000313280803178F00B1
:100090000313290803178C0003132A0803178E0083
:1000A000031320088A00210E8300FF0E7F0E090033
:1000B0008A110A1265298A110A12E8288A110A127D
:1000C00071280D287536F33969106F33E606000084
:1000D0000D2AE51E2532A030F332F43AF31E253204
:1000E0000D0083164C08CC0A193C031879280130FE
:1000F000CB00640083120B118A110A1237284418AE
:100100003018B0366D00412A2B29532A0D05000105
:10011000412AAB214928CD2AD81EB1060A00412A1E
:10012000AB214928D322522B4529BD180D050001CA
:10013000412AAB2157254128BD12E312F312631661
:10014000A531A539A5310D0500014536E939E1256F
:100150006F3AE91B3700CD264C1AB223412A5A1BAD
:10016000C3203200412AAB214928532A4129D41EF9
:100170003116A22A442822162219B51A2E19B51AA8
:100180002E19B51A2E19B51A2216A539AC127316E6
:10019000B2060A00B418B1180001B41831190001F0
:1001A000412AAB21D7264F22C51EB1060A00412A9B
:1001B000AB2149284326CF29C51EB1060A00412A92
:1001C000AB214928D3224E22BD18AC12E4060A0006
:1001D00064000C108A110A1237280317B908031992
:1001E0003A293608FA003508840083137A188317F1
:1001F0000008BA003808FA003708840083137A1818
:10020000831700083A0203191F293608FA00350837
:10021000840083137A1883170008BA003808FA009C
:100220003708840083137A18831700083A020318EA
:100230001B29FF301C290130F8003C292C293608E5
:10024000FA003508840083137A1883178008031D89
:100250002C290030F8003C293608FA003508B50A88
:100260000319B60A3808FA003708B70A0319B80A9A
:10027000B903EE280030F80003130800F701F80175
:1002800003173C0803103D18F707F70CF80CBD18CE
:10029000F707F70CF80C3D19F707F70CF80CBD1928
:1002A000F707F70CF80C3D1AF707F70CF80CBD1A16
:1002B000F707F70CF80C3D1BF707F70CF80CBD1B04
:1002C000F707F70CF80C0313080003171108FA00DE
:1002D0001008840083137A188317B8010408B70044
:1002E0003810831B381403138C1E74291808AC00B3
:1002F0001A08F800AC1C7E291812181603173708C4
:100300008400831338188317780880001108FA00D6
:100310001008900A0319910A840083137A1883172E
:1003200000080A3C031DF82AB6017B30B500B8016D
:10033000CE30B7000230B9000313ED20F8080319DE
:10034000A3290030A4290130F4000317B601B4300A
:10035000B500B801CE30B7000330B9000313ED206B
:1003600078088316EF00EF08031DF22ACD114D081F
:100370008700831287110317B6016930B500B801F1
:10038000D730B7000230B9003608BB003508BA00D4
:10039000B9080319F3293808FA00370884008313D1
:1003A0007A18831780080319F3293B08FA003A08E2
:1003B000BA0A0319BB0ABC007A08BD003808FA0063
:1003C0003708B70A0319B80A840083137A18831709
:1003D0000008BE003C08840083133D1883173E08C4
:1003E0008000B903C829B9080319032A3B08FA0099
:1003F0003A08BA0A0319BB0A840083137A188317D0
:100400008001B903F3293508F8003608F900031311
:10041000EB010317B6016930B500BA01B8010A3023
:10042000B900B70135083604031D192A0030F80059
:10043000EB2A3A08BA0A3507840083133618831763
:100440000008BB003B082D3C031D322A0130B800D8
:100450003A08BA0A35078400831336188317000850
:10046000BB003F2A3B082B3C031D3F2A3A08BA0A2F
:10047000350784008313361883170008BB003B0838
:100480002F3C0318E12A3B08393C031CE12A3B08B6
:10049000303C031D6B2A3A08350784008313361855
:1004A00083170008783C03195F2A3A08350784004F
:1004B0008313361883170008583C031D6B2A10302D
:1004C000B900BA0A3A08BA0A350784008313361805
:1004D00083170008BB0039080A3C031D8F2A3B081C
:1004E0002F3C03188E2A3B08393C031C8E2A0A3005
:1004F000BC003708BD0003133E2178080317BC0079
:1005000030303B023C07B7003A08BA0A350784008E
:100510008313361883170008BB006F2AE12A3908B5
:10052000103C031DE12A3B08603C03189E2A3B084F
:100530007A3C031C9E2A3B08DF399F2A3B08BB00FC
:100540003B082F3C0318A82A3B08393C0318B02A63
:100550003B08403C0318E12A3B08463C031CE12AC7
:100560003B082F3C0318C12A3B08393C031CC12A15
:10057000370EBC00F030BC0530303B023C07B70002
:10058000CA2A370EBC00F030BC0541303B020A3E9F
:100590003C07B7003A08BA0A3507840083133618B7
:1005A00083170008BB003B08603C0318DE2A3B08A9
:1005B0007A3C031CDE2A3B08DF39DF2A3B08BB00FC
:1005C000A02A380BE92A39080A3C031DE92AB70991
:1005D000B70A3708F8007808F30001309300831653
:1005E0000313EF01831203179101CE3090009201A3
:1005F000920A1208203C0318012B9101CE30900082
:10060000920103138C128A110A1237288D192A229B
:10061000D3183819B015C821AD295218B415C529F9
:10062000501C321B36105017D234F430ED30EB34FE
:10063000A018301734173218311B0D00CE32771046
:10064000F332F43AF01E253200001C308400831788
:10065000000803193C2B0230F800BF30F70064009B
:10066000F70B2F2BF80B2D2B9630F700F70B362BB3
:10067000392B6400800B2B2B08000B0803179B0001
:1006800003138B13831603178C170C140000000040
:1006900083129B1F4E2B03138B1703170C087F39F4
:1006A00003198D2B9B000D089C000F089D001B0853
:1006B00003130C1E592B990003171C088D001D08ED
:1006C0008F0003130B0803179E0003138B1383166D
:1006D00003178C170C140000000083129E1F732B4D
:1006E00003138B1703170C0D0E0D7F3903198D2B78
:1006F0009B000D089C000F089D001B0803130C1E97
:100700007F2B990003171C088D001D088F008D0A90
:1007100003198F0A03133D2B0317031308000B085B
:1007200003179D0003138B13831603178C170C14E8
:100730000000000083129D1FA02B03138B170317CB
:100740000318C82B0C087F399D000D089E000F0868
:100750009F001D0803130C1EAB2B990003171E08E6
:100760008D001F088F0003130B080317A00003134D
:100770008B13831603178C170C14000000008312D0
:10078000A01FC52B03138B1703179C0BC82BE32B40
:100790000C0D0E0D7F399D000D089E000F089F0067
:1007A0001D0803130C1ED22B990003171E088D0081
:1007B0001F088F008D0A03198F0A03109C0BE12B71
:1007C000E32B03138F2B0313080064000D300C1E62
:1007D000E72B99000A300C1EEB2B9900F401013035
:1007E0000317950083308D0000308F0003133D23E5
:1007F000831606108312061003179401140F012CA0
:100800000D2CF4080319062C95010B2C14309C00B8
:10081000031325230317940AFE2B9508031DF22BBF
:100820000C309600FA309C00031325230317960B17
:10083000122CF4010130950088308D0000308F00BB
:1008400003133D23031794011408183C031C342C94
:10085000F40803192D2C9501322C14309C0003133D
:1008600025230317940A242C9508031D1C2C023001
:100870009600FA309C00031325230317960B392C9E
:10088000F401013095008F308D0000308F0003138C
:100890003D23031794011408183C031C5B2CF40837
:1008A0000319542C9501592C14309C000313252353
:1008B0000317940A4B2C9508031D432CF4010130B7
:1008C000950098308D0000308F00031009309C0097
:1008D00003138F2322300C1E6B2C9900A5300317B5
:1008E0008D0000308F0003133D2322300C1E762C28
:1008F00099002C300C1E7A2C990022300C1E7E2C74
:100900009900AB3003178D0000308F0003133D2397
:1009100022300C1E892C99000D300C1E8D2C990054
:100920000A300C1E912C9900043003179600FA30FF
:100930009C00031325230317960B972C9401140F87
:10094000A22CAE2CF4080319A72C9501AC2C143062
:100950009C00031325230317940A9F2C9508031D5D
:10096000612CF40101309500B2308D0000308F0011
:10097000031026309C0003138F23CA3003178D0009
:1009800000308F0003133D232C300C1EC52C990022
:10099000CD3003178D0000308F0003133D23C73087
:1009A00003178D0000308F00031404309C000313E4
:1009B0008F23023003179600FA309C00031325237F
:1009C0000317960BDC2C9401140FE72CF32CF4087E
:1009D0000319EC2C9501F12C14309C0003132523F2
:1009E0000317940AE42C9508031DB42CC8309C000E
:1009F00003132523F401013003179500D0308D0037
:100A000000308F0003133D23031794011408183C92
:100A1000031C162DF40803190F2D9501142D143005
:100A20009C00031325230317940A062D9508031D24
:100A3000FE2C03138A110A16A82A83163F08840085
:100A40008313401883178312031728088000840A31
:100A5000800183160313BF0A0319C00A831208001A
:100A60008318352D303084008317F701F801F90120
:100A7000FA010317B001B101B201B3012F082E042E
:100A80002D042C040319742D2030B4000310A80D7C
:100A9000A90DAA0DAB0DB00DB10DB20DB30D2F0800
:100AA0003302031D5D2D2E083202031D5D2D2D081E
:100AB0003102031D5D2D2C083002031C6E2D2C0805
:100AC000B0022D08031C2D0FB1022E08031C2E0F9F
:100AD000B2022F08031C2F0FB3020314F70DF80DF9
:100AE000F90DFA0DB40B462D30088000840A310848
:100AF0008000840A32088000840A330880000313CF
:100B0000080003171C08A0001B089F002008FA001B
:100B10001F08840083137A18831780080319942D03
:100B20009F0A0319A00A862D1E08FA001D088400DA
:100B300083137A18831780080319B72D1F08A100A3
:100B40002008A2001D08840083131E1883170008C4
:100B5000A300210884008313221883172308800030
:100B60009F0A0319A00A9D0A03199E0A942D1F08C3
:100B7000840083132018831780011B08F8001C08C9
:100B8000F90003130800083003179C02031CD42D3E
:100B90001C30840083170310800C00080319D42D27
:100BA000D22D6400800BD12D03130800831605108D
:100BB0000510831205106400023003179B00ED300E
:100BC0009C000313C32503179B0BDF2D8316031310
:100BD000051464002730F700F70BEC2D0000051416
:100BE00083120518032E6400023003179B00ED30BA
:100BF0009C000313C32503179B0BF72D0030F8004F
:100C0000172E172E03136400023003179B00ED30DC
:100C10009C000313C32503179B0B072E61308D0027
:100C200000308F0003133D230130F8000317031336
:100C3000080083160514831203179C011C08073C47
:100C4000031C552E0130F7001C08F80003192C2E48
:100C50000310F70DF80B282E77081B050319432EF8
:100C6000831603130510051083120510640000009D
:100C70008316051464002730F700F70B3D2E0000A3
:100C8000512E8312031783160313051005108312C8
:100C9000051064002730F700F70B4C2E0000831678
:100CA0000514831203179C0A1E2E03130800031752
:100CB0009C01831603130514831203179B011B0861
:100CC000073C031C892E831603130510051083129D
:100CD000051064006B2E00008316051405148312A2
:100CE000051C802E0130F70003171B08F8000319BC
:100CF0007D2E0310F70DF80B792E77089C04031353
:100D000064002730F700F70B832E000003179B0ABF
:100D10005F2E1C08F800031308000317220823069F
:100D20008039A500A21F962EA209A20AA31F9A2EFF
:100D3000A309A30A2308F80122020318A22E2208FD
:100D4000F700AE2EF7010830A400A20DF70D23081E
:100D500077020318F700F80DA40BA52EA51FB22EDD
:100D6000F809F80A03130800083083164A028312B0
:100D700003179C009B1FCC2E83160313410884008D
:100D80008313421883172D308000831203171B082A
:100D9000FF3A013E9B00D72E8316031341088400BF
:100DA00083134218831720308000831203171B0817
:100DB000F7001C08F8000319E12E0310F70CF80BDC
:100DC000DD2E77089D0083160313410884008313EA
:100DD0004218831700082D3C0319152F831203179F
:100DE0001D08A2006430A30003138D2678080319A0
:100DF0000C2F013083164107840083134218831798
:100E0000831203171D08A2006430A30003138D266C
:100E1000303078078000162F013083164107840098
:100E200083134218831730308000831202308316F8
:100E300041078400831342188317831203171D0888
:100E4000A2000A30A30003138D2678080317A2001E
:100E50000A30A30003138D2630307707800003305B
:100E600083164107840083134218831783120317E4
:100E70001D08A2000A30A30003138D263030770727
:100E800080000430831641078400831342188317BF
:100E90002E3080000F30831203179B050313AB0124
:100EA0008B1BAB178B130A300317BC001B08BD004C
:100EB00003133E21AB1B8B17780E03179E000F30D8
:100EC0009E050530831603134107840083134218DF
:100ED00083173030831203171E07800003130800A6
:100EE00003172308F80122020318792F2208F700BC
:100EF000852FF7010830A400A20DF70D2308770213
:100F00000318F700F80DA40B7C2F03130800203002
:100F100003171D1E30309E001C08F7009C1F982FE1
:100F2000F709F70A77089C002D309E009D171D14C5
:100F30001C08A2006430A30003137027770803176E
:100F40009C00303078079F001C08A2000A30A300E4
:100F500003137027303077070317A100303078076C
:100F6000A0001E08F70030301F020319BB2F9D148C
:100F70009D1B1D15CF2F1E089F0020309E00303076
:100F800020020319C72F1D149D1B9D14CF2F031D75
:100F90001D14031DCF2F1F08A00020309F001D1916
:100FA000D62F9D18DC2F1D18E22FE82F1E080313E3
:100FB0000C1ED82F990003171F0803130C1EDE2FD9
:100FC00099000317200803130C1EE42F9900031740
:0C0FD000210803130C1EEA2F99000800F2
:10100000F03097059D05831603170908C03989003C
:1010100003131F129F12003003178800831203135B
:101020001014031787018801890183160313CB016C
:10103000CC014D104D0887008312071464000C305A
:10104000F700F70B2128242883164D104D08870040
:1010500083120710C0308B048316CD144D0887000F
:10106000831287183B288316CB080319392883126B
:101070003B282D2883128E018F018E018316CD14FB
:101080004D0887008312871C4D288316CB0803194F
:101090004B2883124D283F2883120F08FA000E08B0
:1010A000F7000F087A02031D4D28770803179800F0
:1010B0007A0899009A019B0103130B138B138B1B66
:1010C0005E2803171B089F001A089E0019089D0040
:1010D00018089C00B630F700FA01F901F8011C0865
:1010E0001D041E041F04031D7728F7018428031024
:1010F000F81B83289C0D9D0D9E0D9F0DFA0DF90D7B
:10110000F80DF70B7728F8137A089F0079089E00EE
:1011100078089D0077089C00AE30A3004730A200FD
:101120007930A1008230A0001C0803190429A40012
:10113000200803190429A4070318A5287F30A40256
:10114000031C042903190429A9288130A4070318C2
:1011500004292408F700F801F901FA011D08A80084
:10116000A8171E08A7001F08A6001830A400A50194
:10117000261CD2282308FA07031CC428F90A031DD9
:10118000C428F80A0319A5172208F907031CCB285D
:10119000F80A0319A51721089E009E171E08F807D4
:1011A0000318A517A50DF80CF90CFA0CA80CA70C40
:1011B000A60C0310A40BB7280130F7070318042965
:1011C000F81BE928A80DFA0DF90DF80DF70303191E
:1011D0000429A81FFA28FA0A031DFA28F90A031D90
:1011E000FA28F80A031DFA28F80CF90CFA0CF70A89
:1011F000031904291D08A5002108A506A51F022919
:10120000F8170829F8130829F701F801F901FA017C
:101210007A089F0079089E0078089D0077089C0056
:101220001F08A3001E08A2001D08A1001C08A000A2
:10123000A701A6014830A5008530A40020080319A5
:10124000E329AC0024080319E329AC02031C2D296F
:101250007F30AC070318E32933298130AC02031C2B
:10126000E3290319E3292C08F700F801F901FA0131
:10127000AB012108AA00AA172208A9002308A80088
:101280001930AC002708A802031856290130A9021A
:1012900003185629AA0203185629AB020318562927
:1012A000AB0AAA0AA90A2708A80788292608A902BA
:1012B000031871290130AA0203187129AB0203181F
:1012C0007129AB0AAA0A2608A9072708A807031C40
:1012D0008829A90A031D8829AA0A031D8829AB0A9F
:1012E000882925088038AA02031887290130AB0213
:1012F00003188729AB0A25088038AA072608A907FA
:10130000031C6529AA0A031D6529AB0A65297A14FD
:10131000AC0B8B2996290310A80DA90DAA0DAB0DB6
:101320000310FA0DF90DF80DAD0D42292D1C9E2963
:101330000310F80CF90CFA0CAD0CA129F7030319F2
:10134000E329AD1BCA290310A80DA90DAA0DAB0DE9
:101350002708A8020318B6290130A9020318B629E4
:10136000AA020318B629AB02031CD9292608A90230
:101370000318C1290130AA020318C129AB02031CBA
:10138000D92925088038AA020318CA290130AB02DE
:10139000031CD929FA0A031DD929F90A031DD929E1
:1013A000F80A031DD929F70A0319E329F80CF90CE7
:1013B000FA0C2108AC002508AC06AC1FE129F8178F
:1013C000E729F813E729F701F801F901FA017A088A
:1013D0009F0079089E0078089D0077089C00831084
:1013E0001F08A3001E08A2001D08A1001C08A000E1
:1013F0009A30A7009930A6005D30A5008330A40084
:1014000080308318A506AA01AB012108A900250890
:10141000A90620080319F02AA800F70024080319D8
:10142000F92AA8020319952A031C532A2508AE009D
:10143000AE172608AD002708AC00AB010310AE0CB8
:10144000AD0CAC0CAB0CA80B1D2AA91F2A2A2A1420
:101450000D2B2A1028102A16233084008317222BE4
:101460002A12A91B3D2A281C482AAE0CAD0CAC0C34
:10147000AB0CF70A0319082B482AAE1B4B2A0310A2
:10148000AB0DAC0DAD0DAE0DF7030319082B3D2AC6
:101490002A17B52A2A132108A900A91F512AAE1715
:1014A000012BAE13012B2408A800F7002008A80286
:1014B0002108AE00AE172208AD002308AC00AB0136
:1014C0000310AE0CAD0CAC0CAB0CA80B5F2AA91F23
:1014D0006C2AAA140D2BAA102810AA1627308400F3
:1014E0008317222BAA12A91B7F2A281C8A2AAE0C3A
:1014F000AD0CAC0CAB0CF70A0319082B8A2AAE1BF7
:101500008D2A0310AB0DAC0DAD0DAE0DF703031915
:10151000082B7F2AAA17B52AAA132508A900A91FF4
:10152000932AAE17012BAE13012B2508AE00AE1780
:101530002608AD002708AC00A91FA22AAE132A1561
:101540000D2B2A11AB012810233084008317222B86
:10155000A91BCB2A2108A900281CB52AAE0CAD0C6A
:10156000AC0CAB0CF70A0319082BAB1FC62AAC0A4C
:10157000031DC62AAD0A031DC62AAE0A031DC62ACC
:10158000AE0CAD0CAC0CF70A0319082B2A1B4A2A27
:10159000AA1B8C2AEA2A8030AE06AE1FD32A0D2B56
:1015A0002508A900E02A2108A900AE08031DE02AA9
:1015B000AD08031DE02AAC08031DE02AF701012B4A
:1015C000AE1BEA2A0310AB0DAC0DAD0DAE0DF70B43
:1015D000E02A082BA91FEE2AAE17012BAE13012B10
:1015E0002408F7002508AE002608AD002708AC0047
:1015F000012B2008F7002108AE002208AD002308C7
:10160000AC002E08F8002D08F9002C08FA00402B39
:10161000F701F801F901FA01402BAB01AC09AD0962
:10162000AE09AB09AB0A031D1B2BAC0A031D1B2B18
:10163000AD0A0319AE0A2A18292AAA186B2A2A19F0
:10164000A12AD02A0008AC07031C2C2BAD0A031DCD
:101650002C2BAE0A0319281484030008AD07031CC1
:10166000342BAE0A0319281484030008801F803A23
:10167000AE07031828142A1A302AAA1A722AA82A8E
:101680007A089F0079089E0078089D0077089C00E2
:101690001C08B63C9C00FA011D08A0009D17031011
:1016A0009D0C9E0C9F0CFA0CF90CF80CF70C9C0B83
:1016B0004F2BA01F662BF709F809F909FA09F70A59
:1016C0000319F80A0319F90A0319FA0A7A089700A4
:1016D0007908960078089500770894009B08031D08
:1016E0000B2C9A08031D0B2C1908323C031C0B2CE5
:1016F000031D7E2B1808C73C031C0B2C83160313F9
:10170000C0012D30BF00443083120317A8008A1196
:1017100003131D258A1544308400031717089F0002
:1017200016089E0015089D0014089C000408A000DF
:101730003B30A7009A30A600CA30A500A4010A30A9
:10174000A20083141C30840083171F08AB001E08FE
:10175000AA001D08A9001C08A8002708AF00260839
:10176000AE002508AD002408AC008A110313302513
:101770008A157808F708031DD42B03172208013AAD
:10178000031DC42B0313D42B20080319D62B0F39A8
:1017900022020319CD2B0318DF2BA01BDF2B201BEC
:1017A000D62B2030D72B03130317A0013030F707B7
:1017B0007708A8008A1103131D258A1503178310C3
:1017C0002708AB002608AA002508A9002408A800BD
:1017D000AF01AE01AD010A30AC008A110313302510
:1017E0008A157A080317A7007908A6007808A500CB
:1017F0007708A400A20BA12B6D30A8008A11031357
:101800001D258A156D300317A8008A1103131D25A5
:101810008A15682C031783160313C0012D30BF00EF
:101820007F30831203178D0000308F0003130B08E5
:1018300003179C0003138B13831603178C170C14C8
:101840000000000083129C1F282C03138B17031722
:101850000C087F390319672C9C000D089D000F08A8
:101860009E001C08A8008A1103131D258A15031762
:101870001D088D001E088F0003130B0803179F001F
:1018800003138B13831603178C170C14000000002E
:1018900083129F1F4E2C03138B1703170C0D0E0D75
:1018A0007F390319672C9C000D089D000F089E00CE
:1018B0001C08A8008A1103131D258A1503171D088B
:1018C0008D001E088F008D0A03198F0A162C031332
:1018D0008A110A16BA2A203003171C1E30309D00C8
:1018E0001B08F7009B1F7C2CF709F70A77089B0061
:1018F0002D309D009C171C141B08A2006430A3000F
:101900008A11031370278A15770803179B0030305C
:1019100078079E001B08A2000A30A3008A11031357
:1019200070278A15303077070317A000303078070A
:101930009F001D08F70030301E020319A32C9C14D1
:101940009C1B1C15B72C1D089E0020309D003030BC
:101950001F020319AF2C1C149C1B9C14B72C031DD5
:101960001C14031DB72C1E089F0020309E001C195C
:10197000BE2C9C18C52C1C18CC2CD32C1D08A800E0
:101980008A1103131D258A1503171E08A8008A1142
:1019900003131D258A1503171F08A8008A110313B6
:1019A0001D258A1503172008A8008A1103131D2579
:1019B0008A15080080080319F82C03179C010408F5
:1019C0009B001C10831B1C140008A8008A11031321
:1019D0001D258A1503171B08840083131C18831701
:1019E000840A031DF62C0313850A03170313DA2C4C
:1019F000080083164108840083134218831780016E
:101A00003030831203179400950096002E30970013
:101A1000303098009901831603134208831203178C
:101A20009C00831603134108831203179B000130A7
:101A30009E0014309D008A11031381258A1564309D
:101A400003179C008A11031325238A158A11D625B2
:101A50008A15F808031DC92DCC3003179B008A1185
:101A6000031319268A15443003179B008A110313A8
:101A700019268A15033003179B00FA309C008A113F
:101A8000031325238A1503179B0B3D2D8A1103137E
:101A9000D6258A15CC3003179B008A11031319260B
:101AA0008A15BE3003179B008A11031319268A1565
:101AB0008A1157268A1578088316BE008A11831268
:101AC00057268A1500308316BE073E088312031777
:101AD0009B008A110313B4268A1583163E088312CD
:101AE0000317A2000230A3008A1103138D268A1562
:101AF000780803179B0068308D0000308F000310BA
:101B000004309C008A1103138F238A1503171B08C6
:101B10009C0018309D008A11031387278A156B30AB
:101B200003178D0000308F00031008309C008A11CD
:101B300003138F238A15730803179C0018309D0028
:101B40008A11031387278A150D300C1EA52D9900C5
:101B500083163E0883120317A2000230A3008A11E5
:101B600003138D268A15F81BB92D73087802031804
:101B7000C22D013003179A00831603130610831237
:101B80000614C92D831606108312061003179A0136
:101B900003138316C0014130BF007308831203177B
:101BA0009B0001309C0020301C1E30309D001B0823
:101BB000F7009B1FE32DF709F70A77089B002D30EC
:101BC0009D009C171C141B08A2006430A3008A11FE
:101BD000031370278A15770803179B0030307807A6
:101BE0009E001B08A2000A30A3008A11031370276D
:101BF0008A15303077070317A000303078079F0030
:101C00001D08F70030301E0203190A2E9C149C1B7D
:101C10001C151E2E1C191E2E1D089E009C18152E0C
:101C200030301F020319182E1C149C1B9C141E2EEE
:101C3000031D1C14031D1E2E1E089F001C19252E9B
:101C40009C182C2E1C18332E3A2E1D08A8008A1121
:101C500003131D258A1503171E08A8008A110313F4
:101C60001D258A1503171F08A8008A1103131D25B7
:101C70008A1503172008A8008A1103131D258A1549
:101C800003171A089B0018309C0003136B24433081
:101C90000317A8008A1103131D258A153030031776
:101CA000A8008A1103131D258A155F300317A800A9
:101CB0008A1103131D258A1583163F088400831398
:101CC000401883178001410884008313421883174A
:101CD0008312DA248A110A16CA2A831685108510FF
:101CE000831285106400023003179A00ED309C00C7
:101CF0008A110313C3258A1503179A0B762E8316B0
:101D00000313851464002730F700F70B852E0000BD
:101D10008514831285189E2E6400023003179A00E2
:101D2000ED309C008A110313C3258A1503179A0B03
:101D3000902E0030F800AD2EAD2E0313640002305B
:101D400003179A00ED309C008A110313C3258A15EE
:101D500003179A0BA22E0130F80003130800831614
:101D60008514831203179B011B08073C031CEC2EF0
:101D70000130F7001B08F8000319C22E0310F70DFD
:101D8000F80BBE2E77081A050319DA2E83160313F3
:101D900085108510831285106400CE2E00008316F6
:101DA000851464002730F700F70BD42E0000E82ECE
:101DB0008312031783160313851085108312851071
:101DC00064002730F700F70BE32E0000831685141C
:101DD000831203179B0AB42E0313080003179B01F9
:101DE000831603138514831203179A011A08073CFC
:101DF000031C202F83160313851085108312851072
:101E00006400022F00008316851485148312851C3C
:101E1000172F0130F70003171A08F8000319142FC1
:101E20000310F70DF80B102F77089B0403136400C1
:101E30002730F700F70B1A2F000003179A0AF62E27
:101E40001B08F8000313080083164108840083135D
:101E500042188317800130308312031794009500D5
:101E600096002E30970030309800990183160313A6
:101E70004208831203179C00831603134108831240
:101E800003179B0001309E0014309D008A1103133C
:101E900081258A156D26F808031D832FCC30031782
:101EA0009A000313AF26443003179A000313AF269A
:101EB000033003179A00FA309C008A11031325237C
:101EC0008A1503179A0B5B2F03136D26CC3003176B
:101ED0009A000313AF26BE3003179A000313AF26F0
:101EE000EE2678088316BE008312EE260030831695
:101EF000BE077830BE023E08831203179B008A118A
:101F00000313B4268A158316C0015530BF00433031
:101F100083120317A8008A1103131D258A15313077
:101F20000317A8008A1103131D258A155F300317B4
:101F3000A8008A1103131D258A1583163F08840003
:101F400083134018831780014108840083134218CB
:101F500083178312DA248A110A16DA2A83160511E6
:101F60000511831205116400023003179A00ED3049
:101F70009C008A110313C3258A1503179A0BB72FE8
:101F800083160313051564002730F700F70BC62FDF
:101F90000000051583120519DF2F640002300317B6
:101FA0009A00ED309C008A110313C3258A1503178C
:101FB0009A0BD12F0030F800EE2FEE2F03136400A0
:101FC000023003179A00ED309C008A110313C325D9
:101FD0008A1503179A0BE32F0130F800031308004A
:1020000083160515831203179B011B08073C031C4D
:102010003C280130F7001B08F800031913280310AF
:10202000F70DF80B0F2877081A0503192A288316CD
:1020300003130511051183120511640000008316B6
:10204000051564002730F700F70B24280000382816
:10205000831203178316031305110511831205114B
:1020600064002730F700F70B3328000083160515AE
:10207000831203179B0A05280313080003179B010B
:10208000831603130515831203179A011A08073CD8
:10209000031C702883160313051105118312051103
:1020A0006400522800008316051505158312051DCE
:1020B00067280130F70003171A08F800031964288D
:1020C0000310F70DF80B602877089B0403136400D6
:1020D0002730F700F70B6A28000003179A0A4628F2
:1020E0001B08F800031308008316410884008313BB
:1020F0004218831780013030831203179400950033
:1021000096002E3097003030980099018316031303
:102110004208831203179C0083160313410883129D
:1021200003179B0001309E0014309D000A12031318
:1021300081250A160A128A15AE270A168A11F8088E
:10214000031DD928CC3003179A0003130020443014
:1021500003179A0003130020033003179A00FA3084
:102160009C000A12031325230A1603179A0BAF28A3
:102170000A128A150313AE270A168A11CC300317E8
:102180009A0003130020BE3003179A0003130020A7
:102190003E2078088316BE0083123E20003083164E
:1021A000BE073E08831203179B000A120313B426CE
:1021B0000A168316C001A030BF00433083120317F4
:1021C000A8000A1203131D250A1632300317A800AF
:1021D0000A1203131D250A165F300317A8000A12FE
:1021E00003131D250A1683163F0884008313401825
:1021F00083178001410884008313421883170A1251
:102200008A158312DA240A168A118A110A16E82A14
:102210008316CD114D088700831287150317150803
:1022200098001408970018089A00170899001A08CF
:10223000FA001908840083137A1883178008031999
:102240002529990A03199A0A172917081902F7006C
:102250001A08FA001808031C180FFA027708F80089
:1022600078089600DF308D0000308F0003100D30AD
:102270009C000A1203138F230A16031716089C00EA
:1022800018309D000A12031387270A160D300C1E02
:10229000472999000A300C1E4B2999006430031716
:1022A0009C000A12031325230A160317140884003E
:1022B00083131518831780080319762998010408D9
:1022C00097001810831B1814000803130C1E6629AE
:1022D0009900031717088400831318188317840ABA
:1022E000031D75290313850A03175B2903130800CF
:1022F0000B080317950003138B13831603178C1712
:102300000C14000000008312951F892903138B17FA
:1023100003170318B2290C087F3995000D089600A1
:102320000F0897001508A8000A1203131D250A16A6
:10233000031716088D0017088F0003130B080317E7
:10234000980003138B13831603178C170C140000CB
:1023500000008312981FAF2903138B170317940BE8
:10236000B229CE290C0D0E0D7F3995000D0896006F
:102370000F0897001508A8000A1203131D250A1656
:10238000031716088D0017088F008D0A03198F0A8E
:102390000310940BCC29CE290313782903138A1137
:1023A0000A160F2B03081F398300713083168F0024
:1023B00090010F088312AC018316031787151030A4
:1023C0000313990000309A00A630980090308312D1
:1023D00098001430F300F4018316C001BF010930E6
:1023E000CA00FF30CD00EF01831203179201930161
:1023F00083160908C039890003131F129F12003089
:1024000003178800831287018801890183136B30C9
:102410000313AD006F30AE006530AF00B0012B305C
:102420008316B4004930B5005030B6004430B700D0
:102430002C30B800B9014F30FB004B30FC00FD01DF
:10244000F501F6013030C300C400C500C6002E30CF
:10245000C7003030C800C901C201C330C1006400E8
:1024600006108312061403179101CE3090008316D4
:1024700003130E120D3083120C1E3C2A9900643097
:1024800003179C000A12031325230A1606300317AC
:102490008D0003308F000A1203133D230A166430A7
:1024A00003179C000A12031325230A168316031729
:1024B0000908C039890003131F129F120030031747
:1024C0008800831203131F179F1783169F17831209
:1024D0001F14F8001F08C33978049F006400831696
:1024E0000108C039810035308312900083160C1426
:1024F00083128B1683168C16C03083128B0403173D
:102500008D0183168C130C1483120C08F300043015
:102510009400FA309C000A12031325230A160317AD
:10252000940B892A83160313CD114D08870083125B
:102530008715043003179400FA309C000A12031325
:1025400025230A160317940B9C2A0A120313E52B62
:102550000A16640083168C12CD114D088700831271
:102560008715AD01C101D5018316A0010A128A1594
:10257000831200280A168A110B138B138B1BBD2A9A
:10258000643003179C000A12031325230A160A124B
:102590008A15F92C0A168A1103179C012D309B000D
:1025A0009E0141309D000A12031381250A160A126A
:1025B0008A15242F0A168A1103179C012D309B00BF
:1025C0009E0155309D000A12031381250A167428B6
:1025D00003179C012D309B009E01A0309D000A1224
:1025E000031381250A16031795012D309400031358
:1025F0000821C0308B04031793080319522B83164C
:102600000313C0012D30BF001E30831203178D004D
:1026100003308F0003100A309400031378297308E5
:1026200003179B0018309C000A128A1503136B24B1
:102630000A168A11031795012D30940003130821FF
:102640000317930103130B08F7008B1303178D0176
:1026500073088C0083168C130C1555308D00AA302E
:102660008D008C148C18322B0C11770883120313F5
:102670008B048316CD114D088700831287158316AE
:10268000CE01831203179101CE30900092010C30DD
:102690009400FA309C000A12031325230A1603172C
:0A26A000940B492B0313A92A6300D1
:024200001B00A1
:04400E00C42D0006B7
:00000001FF
